:0C00000020C0FECFFDCFFCCFFBCFFACF1D
:10000C00F9CFF8CFF7CFF6CFF5CF44C0F3CFF2CF7F
:10001C00F1CFF0CFEFCFEECFEDCF1027E803640098
:10002C000A00010000100001100001000000010096
:10003C00050038000000F894EE27ECBBF1E0FBBFA4
:10004C00EBBFE5BFF8E1F1BDE1BD8DE0A2E0BB2760
:10005C00ED938A95E9F780E094E0A0E6ED930197A3
:10006C00E9F7EAE3F0E085919591009761F0A591AD
:10007C00B59105901590BF01F00105900D92019777
:10008C00E1F7FB01F0CFEFE5EDBFE4E0EEBFC0E63A
:10009C00D1E066C00A921A92FA926A937A938A9382
:1000AC009A93AA93BA93EA93FA93EFB7EA931A93B3
:1000BC001CB1E0E0E51511F4133209F004C06BD16A
:1000CC00E1E05E2E3EC0E6E05E1618F464D1539477
:1000DC0038C01D30B1F55524E091610162D13097E3
:1000EC0069F461D17F936F93FF93EF936DD1AF91CF
:1000FC00BF918F919F9171D1EAE221C0E130A0E0D4
:10010C00FA0769F450D17F936F93FF93EF935CD10F
:10011C00AF91BF918F919F9160D1E2E310C0E2301B
:10012C00A0E0FA0771F43FD17F936F93FF93EF93A5
:10013C004BD1AF91BF918F919F914FD1EAE3EA934D
:10014C002BD01991E991EFBFF991E991B991A9914E
:10015C009991899179916991F990199009901895D3
:10016C00E6D085D0FFCFFFCFE4EAE6BFE6B7E7FFE6
:10017C00FDCFE0EC3CD1E6B7E7FFFDCFE98137D10D
:10018C00E6B7E7FFFDCFE88132D1E6B7E7FFFDCF59
:10019C00E4E9E6BF229608952497E0E0E883E9833A
:1001AC00EA83EB8328D12CD148F025D1A138E1ED9D
:1001BC00BE07E0EF8E07E8E09E0708F01FC028D1CD
:1001CC00A0E0B9EE84EA95E3A4D1A0E8B0E080E029
:1001DC0090E07FD122D111F4E0E10BC0E233A0E03A
:1001EC00FA0711F4E1E105C0EA33A0E0FA0721F4C3
:1001FC00E2E1EA931DD1B8DF1ED11DC0FCD000D1C5
:10020C00A0F506D1A0E0B6E483EC93E282D105D14F
:10021C0011F4E0E10BC0E233A0E0FA0711F4E1E1E4
:10022C0005C0EA33A0E0FA0721F4E2E1EA93EFE239
:10023C0016D101D1E067EA9397DFEC81ED5FEA9389
:10024C00A981BA818B819C81E8E028D108D1EC810D
:10025C00EC5FEA93E98103D1EC81EB5F02D1EC8195
:10026C00EA5FFFD0EC81E95FFCD029960895E8E1C4
:10027C00EA93E5E1F4D0E3E0EA93EFEFF0D0E0E1CC
:10028C00F3D0E1E1F1D0E2E1EFD0E2E0EDD0D0D07B
:10029C00E0E0E5D0E0E1EA93CBD066DFE1E1EA9380
:1002AC00C7D062DFE2E1EA93C3D05EDFEAE1D9D0E6
:1002BC00EBE1EA93E1E0D3D0ECE1D3D0EDE1EA93CA
:1002CC00E0E1CDD0EEE1CDD0EFE1CBD0E0E2C9D092
:1002DC00E1E2C7D0E2E2C5D0E3E2EA93E1E0BFD0CD
:1002EC00E4E2BFD0E5E2EA93EAE0B9D0E6E2B9D0C5
:1002FC00E7E2B7D0E8E2B5D0E9E2B3D0B8D0EAE2B1
:10030C00EA934ADFB4D0E2E3EA9346DFB0D0EAE303
:10031C00EA9342DFE7EBEA93E2E9A1D0E1EBEA935F
:10032C00ECEA9DD0E3E0EA93E8EF99D00895E0E0A1
:10033C00E8BBE7BBE5BBE4BBE2BBE4E0E1BBE0E070
:10034C00E3BFE2BFEFBDEEBDEDBDECBDE7BDE6BD6D
:10035C00EBBDEABDE9BDE8BDE2BDE5BDE4BDE3BD75
:10036C00E5BFE9BFEBB9E8E9EAB9E6E8E0BDE0E0F2
:10037C00E0BDE7E6E9B9E0E8E8B9E0E0E0BFE6B9FE
:10038C00EDB9ECE0E0B9E0E0E2B9E4E0E6BFE0E0D2
:10039C00E1B978940895E52DF0E0E05AFE4F108312
:1003AC000895F0E00895E0916201FBDF8DD0DF014C
:1003BC00CB01E8E167D0DF01CB01E0916301F1DF14
:1003CC0083D07DD05AD00895E0916401EADF7CD0CF
:1003DC00DF01CB01E8E056D008954FD0DF01CB010F
:1003EC00E0916501DEDF70D048D0BDD00895E3B94F
:1003FC00E4E8E6BF0895AD81BE818F8198850895AC
:10040C00A034E2E4BE07EFE08E07E0E09E0708951B
:10041C00ED81FE816F8178850895E050F240604057
:10042C0070409CD0EC81BDDFEA32A0E0FA07089561
:10043C00EFE0EA930895EC81EA93E0E0EA9394DE2E
:10044C00EC81EF5FEA93E1E0EA938EDEEC81EE5F04
:10045C00EA93E981FA816B817C812CD00895EA932F
:10046C0083CEEA93E0E0FBCFEA93E0E8F8CFE0E458
:10047C00F2E46FE070E077D00895EA2BFB2B682B49
:10048C00792B0895EE230E2EFD01BC0131F0EE0FF9
:10049C00FF1F661F771F0A94D1F70895EE230E2EC7
:1004AC00FD01BC0131F076956795F795E7950A94B7
:1004BC00D1F70895E62FF72F60E070E008956E2FC6
:1004CC007F2FE0E0F0E008956F2F660F660B762F1C
:1004DC0008957A9F702D6B9F700DF89F700DE99F9A
:1004EC00700D6A9F602D710DFB9F600D711DE89F53
:1004FC00600D711D8827FA9FF02D610D781FEB9F01
:10050C00F00D611D781FEA9FE02DF10D681F781F1B
:10051C0008953F934F935F9300241124442755274C
:10052C0030E2AA0FBB1F881F991F001C111C441F0F
:10053C00551F0E1A1F0A460B570B28F40E0E1F1EC2
:10054C00461F571F01C0A1603A9559F7FD01BC0128
:10055C00D001CA015F914F913F910895E883F983CF
:10056C006A837B8308957A936A93FA93EA93089546
:00000001FF
